:020000040000fa
:08000000a2060400000000004c
:020000040000fa
:020000040002f8
:04afe000dfff00008f
:020000040000fa
:020000040002f8
:04afe400ffff00006b
:020000040000fa
:020000040002f8
:04afe80078ff0000ee
:020000040000fa
:020000040002f8
:04afec007dff0000e5
:020000040000fa
:020000040002f8
:04aff00078ff0000e6
:020000040000fa
:1000080000000000000000000000000000000000e8
:100018009a06000000000000000000000000000038
:1000280000000000000000000000000014090000ab
:1000380000000000000000000000000000000000b8
:10004800560900000000000000000000e009000060
:100058004c0a0000780a00000000000000000000c0
:100068000000000000000000000000000000000088
:100078000000000000000000000000000000000078
:1000880000000000000000000000000082090000dd
:10009800b00900000000000000000000000000009f
:1000a8000000000000000000000000000000000048
:1000b8000000000000000000000000000000000038
:1000c8000000000000000000000000000000000028
:1000d8000000000000000000000000000000000018
:1000e8000000000000000000000000000000000008
:1000f80000000000000000000000000000000000f8
:1001080000000000000000000000000000000000e7
:1001180000000000000000000000000000000000d7
:1001280000000000180a00000000000000000000a5
:1001380000000000000000000000000000000000b7
:1001480000000000000000000000000000000000a7
:100158000000000000000000000000000000000097
:100168000000000000000000000000000000000087
:100178000000000000000000000000000000000077
:100188000000000000000000000000000000000067
:100198000000000000000000aa0a0000d60a0000c3
:1001a800020b00000000000000000000000000003a
:1001b8000000000000000000000000000000000037
:1001c8000000000000000000000000000000000027
:1001d8000000000000000000000000000000000017
:1001e8000000000000000000000000000000000007
:1001f80000000000000000000000000000000000f7
:1002080000000000000000000000000000000000e6
:1002180000000000000000000000000000000000d6
:1002280000000000000000000000000000000000c6
:1002380000000000000000000000000000000000b6
:1002480000000000000000000000000000000000a6
:100258000000000000000000000000000000000096
:100268000000000000000000000000000000000086
:0c0278000000000000000000000000007a
:020000040000fa
:10040000803e2000030007008100e900fcff3a0065
:1004100000000600831f7800c20320000400bc0017
:1004200066015100e0815900f23fb1000380b10044
:1004300006003500ee03090000000000423fb10055
:100440000380b100fbff3d001200b000223fb0006e
:10045000020035000280090000000000cf01780092
:10046000000006000001eb00869fbe00889fbe00d2
:100470008a9fbe008c9fbe00820578000004be00eb
:10048000e00107000800be006420e1000700390019
:1004900002003a00f1ff2f00f0ff27000160a000ea
:1004a0001202200012918800560037006120e100fe
:1004b00003003a000b00a70001f8230051003700a9
:1004c00001f0a10002002100936424005200070003
:1004d0000800be0005003500b2fd2000930c24008a
:1004e00004002000690007000004be000005eb00c6
:1004f0000b00a6004f0dde0001f0a1000004be00bd
:1005000032982f0023ea23000f0107000001eb00bf
:10051000030020000b00a70003f82300ac00070035
:100520003e0107000000a7000a00a20080010700aa
:100530000b00e000030032000200200003f0230063
:10054000a200070001f0a2000006be000200200089
:1005500093042400fc0007000801be009c00070073
:10056000809fbe000c00be0022a22a00d3a7230059
:10057000f50007004f01be00950007000004be0013
:1005800001f0a100020020000398230022000700d0
:100590000800be00190035000001be00ea00070097
:1005a0000006be00b2c52900e3622300e600070092
:1005b00022222b00f3942b00850007000c01be00c3
:1005c000e1000700e273280083c0230080000700d9
:1005d0000c01be00dc00070042aa2a00a3e22b00a7
:1005e0007b0007000c01be00d70007000801be0019
:1005f000d50007000801be00750007000a00a7002b
:1006000001f0a2004f06be004f05be004f04be0021
:100610004f03be000000060014002000889fbe00ab
:100620008a9fbe00841f78006e0107004f0078008b
:1006300011003300f0ff2f00838f6c0006003b0099
:10064000040565000a00a7000800370009f0a600ad
:100650001000200008003700820f5400838f5c00d8
:10066000030039001000200001003e0000002000bf
:1006700009f0a7000000ea004f05be004f04be00cd
:100680000000e0000000060014002000869fbe006d
:10069000889fbe008a9fbe008c9fbe004f26dd0053
:1006a00050010700920133006120e1004300320055
:1006b0006250e10041003e003e0039006420e1004c
:1006c0003c003200058255000f003b000402e800a8
:1006d00038003a00800f5300818f5b0035003400f2
:1006e0000800be0003f0a10001f0a60003f0a00086
:1006f0000cf0a70036000700860137000603430010
:1007000087834b000c4646000005530081855b0043
:10071000020033000a03be000c00a0000402e9003e
:10072000f6ff3b00850578000602430087824b00f8
:1007300004003a006000b80009f0a70001f0a00032
:10074000740137000002520081825a000704e00061
:10075000040033000603430087834b008b05e90048
:10076000faff3700090578000604be000203be0048
:100770006011b80038010700e00f5200e08f5a0006
:100780000700350002003c000c08a3000400320002
:100790000601be0003f0a0000cf0a7000c0007004b
:1007a0000a85680001f0a1000af0a70001f0a0008e
:1007b000580137000800be00560137001002200023
:1007c0000cf0a600109188005701370003f0a2003a
:1007d000869fbe00889fbe008a9fbe008c9fbe0081
:1007e00000010700420133006450e1004f00320075
:1007f0006420e1005200320003826c0007003b00dd
:100800000905d0000306d000820f54000c065d00dd
:1008100002003900020032008901780003067800e6
:100820008582550004003d000003fd008103fd00aa
:100830008502ea008b854200840f720002003b00b3
:1008400060001000e08018006011b8000005eb00a7
:100850007a28e1000a00390006007800c75ddd0053
:10086000f707b200878075002d0037008281710084
:100870000a017800610560008180d1000080d3000a
:100880008502e900f9ff3b00060440008784480028
:1008900002003b0060041400e0841c000988a300ef
:1008a000070032008a817100828171006101640059
:1008b0008904d1000884d3008b05e80017003700b5
:1008c0000978a30013003a000b00e0001300340085
:1008d0008b05e9000804440089844c000a44740034
:1008e0000978a3000d003a000b00e0000700340077
:1008f0008b05e9000804440089844c0001003a009b
:100900000b0020000978a300f7ff32000001eb0084
:1009100002003700828171000a017800ce000700d2
:100920000cf0a70001f0a000fa0037006420e100fd
:1009300002003a00838f6c00fb0033000801be0008
:100940000200be00f3003700869fbe00889fbe00f5
:100950008a9fbe008c9fbe00a2000700e400330007
:1009600003866c006450e100240032006420e10042
:10097000270032006150e100220032006120e100d6
:10098000210032008b854200eb07b1000134b80032
:10099000003ab8000804420089844a00013ab800cd
:1009a0000030b8008880400009014a00040033008c
:1009b0000000400081804800020149008b05e900e9
:1009c000c909dd008301700001003200130020001e
:1009d000c814de004814dd004709de001200b20032
:1009e000c808de00088470009b00070001f0a10029
:1009f0000cf0a70001f0a000c60037006120e10064
:100a0000c90032000801be000200be00f7ff370037
:100a10006150e100fcff3a00c3003700829fbe0036
:100a20000001be00770007000470a70003f0a100da
:100a30006509b100180032000e0035006828e10099
:100a400007003500f0ff2f00f1ff27000300e00052
:100a500015003b00010028004f01be00000005000a
:100a600000004000818048008502e900fcff3a0058
:100a700009003700f88f420003003c008000eb00c3
:100a80004f01be00000005008100d1000080d300ae
:100a90008502e800fcff3a000300e00002003b0092
:100aa00060001000e08018004f01be00000006004a
:100ab000829fbe000001be00520007000470a70024
:100ac00003f0a10003f8a30015003a006509b10086
:100ad000110032000a0035006928e10003003500ea
:100ae000010028004f01be0000000500000040008a
:100af000818048008502e900fcff3a0006003700cb
:100b0000f88f4200060035008100d1000080d3003c
:100b10008502e800fcff3a004f01be00000006001d
:100b20008000eb004f01be00000005008000eb00dc
:100b3000829fbe00889fbe008a9fbe00010578008c
:100b40000100e0000400350008003c000000e00067
:100b5000200032000500370060001000e08018001f
:100b600002003b0001f024001a0037000004be0020
:100b70006011b8006b0920000982cf000200390023
:100b80000882cf000441b000694252000e003200da
:100b900008003b0082817100610164008904d1007a
:100ba0000884d3008b05e8000442e800f9ff3a000e
:100bb000050037000804440089844c008b05e900d7
:100bc0000442e900fbff3a00230007000af0a700f7
:100bd00001f0a0004f05be004f04be004f01be0053
:100be000000006000004be00060007000003be006f
:100bf0000405be000200be0002000700844f75001d
:100c000000000600c70ade00f107b200f50fb200cf
:100c100008003200e1cf4200020032000170a00063
:100c200024000500810f7000010032000408050057
:100c300044000500810f700002003a001400050016
:100c40008502e9000000400081c04800fcff3b0035
:100c50000170a00024000500810020006180550083
:100c60000b003d000b00200061fe2f000100e100a1
:100c70001d00340082817100610164008904d1008b
:100c80000884d3000000e800faff3a007100200059
:100c9000610064000300700002006000090032007f
:100ca00061044400e0844c000988a500050032007e
:100cb0008b05e8006808e10002003a008904d100d1
:100cc0000884d300f20f20000258e10005003d0027
:100cd000c75ddd00f907b200898075000800780063
:100ce000000006000bf827008b00780000000500cc
:100cf0000200be006450e100050036006420e100ff
:100d0000020036000968a30001003a000800be0096
:100d10000160a0004f06be004f05be004f04be009c
:100d20004f03be0000000600f0ff2f00f1ff270078
:100d3000f8ff37000020ef000220ef00c088a90074
:100d4000004006000f002100b02e210000018800a5
:100d5000000000000000eb00000778000c00090014
:100d6000002f78000007eb005420ef000e2eef005c
:100d70001e2eef000000eb00a1212100e51d09005f
:100d80008018780040a7a900a10020009cfd070062
:100d9000e0022000303a880044e7a90044c7a900d7
:100da0004407a9004427a9004447a9004467a900b3
:100db0004487a900300020000600fc0031742000a8
:100dc00082072000a3092000824878008348780029
:100dd00080487800113a8000618070000600fc00b5
:100de00021742000620420007305200082487800ee
:100df00083487800804878004427ef00e002200014
:100e0000303a8800300020000d00fc0031742000d2
:100e100082072000a30920008248780083487800d8
:100e20008048780000002000217420006204200027
:100e30007305200082487800834878008048780055
:100e400042a7ae00feff3700813e20006cfd070088
:100e500010c0b30086e6b70090c2b300c4e6b70086
:100e60001002200000708800007825008070880043
:100e700010aea90010cea900102ea900002ea900c6
:100e8000100ea9006004070046050700660607006b
:100e9000440607000000eb00c1762100ff000900b6
:100ea000805878004a72ef004b72ef003632ef0044
:100eb0003832ef000080eb0081762100010009004c
:100ec000801878002832ef0010cea90014cea900b7
:100ed0006632a9003232ef004188a80041a8a9007b
:100ee00041c8a80000a1ef000058220010088800a7
:100ef00004a1a8000481a90005e1a8000068a900d8
:100f00002068a8001061a8001021a90011e1a80024
:100f100011a1a90010a1a8001081a8000621ef00ce
:100f20000a21ef000ca1ef000ea1ef004408a90078
:100f30004428a9004448a9000108a9002108a800e4
:100f400021e1a80021a1a90020c1a90020a1a80099
:100f50002081a8002021a9004e08a8004e28a90041
:100f60004e48a8000388a90040922000e0088800ad
:100f70002388a8002002a9002022a9002042a9005d
:100f800020a2a9002062a9002082a90020e2a900d5
:100f90002102a9002122a900700720004011880029
:100fa00022a2a90022c2a90022e2a90021e2a800ef
:100fb0002182a9004588a90045a8a80045c8a80025
:100fc0002168a8002828a8000e0ea80021e3a90087
:100fd0002143a80021a3a9002123a9002103a900de
:100fe00020e3a80020c3a80020a3a8002083a90014
:100ff0002043a90023e3a90023c3a90023a3a90038
:101000002343a9002323a9002303a90022c3a90085
:1010100022a3a9002283a9002263a9002243a900d8
:101020002223a9002203a9002563ef0024e3ef0097
:101030003223ef002823ef002623ef002e23ef00ba
:101040003023ef0021a8a80001a8a90021e3a800ef
:101050002008a8000008a900c208a9002bc8a90000
:101060002be8a9002c08a9000bc8a9000be8a900cf
:101070000c08a90001eca90001aca900016ca900b1
:10108000014ca900012ca900010ca90000eca90049
:10109000008ca90000aca90000cca900000ca9009c
:1010a000002ca900004ca900006ca900202cef0026
:1010b000402cef00602cef00001020002060880022
:1010c000020ca900022ca800024ca800f007200086
:1010d00030618800f007200030628800f0072000af
:1010e00030638800282cef00482cef00682cef00bc
:1010f000001020005060880023eca80023cca8003a
:1011000023aca900238ca900236ca900234ca800c0
:10111000232ca900230ca900222ca90043eca80031
:1011200043cca80043aca900438ca900436ca900a0
:10113000434ca800432ca900430ca90063eca80071
:1011400063cca80063aca900638ca800636ca90001
:10115000634ca800dabc2a001b32240030002c00ab
:10116000fa608800fb60880020618800dabc2a00f1
:101170001b32240000402c00fa608800fb608800cd
:1011800010618800dabc2a001b32240030002c00d9
:10119000fa608800fb60880020628800dabc2a00c0
:1011a0001b32240000402c00fa608800fb6088009d
:1011b00010628800dabc2a001b32240030002c00a8
:1011c000fa608800fb60880020638800dabc2a008f
:1011d0001b32240000402c00fa608800fb6088006d
:1011e00010638800218ca900418ca900618ca900a2
:1011f000216ca900416ca900616ca900214ca900d7
:10120000414ca900614ca90020eca80040eca800ca
:1012100060eca8003e2cef005e2cef007e2cef006f
:1012200001eca80019013700ff3ffc004200f80064
:101230003600f8004400f8008e1f78000e002000f1
:101240000d000900be1f78003200f8000100fc000c
:101250000068a9000021ef002bd2bf000080fb0036
:10126000306188002dd2bf000080fb003062880012
:101270002fd2bf000080fb00306388005e72ec005c
:10128000ff3ffc003200f900ae0120000d00090014
:101290004f1778004f0778004400f9003600f90036
:1012a0004200f9000100fc0000400600ff3ffc0086
:1012b0004200f8003600f8004400f8008e1f780065
:1012c0000e0020000d000900be1f78003200f8005b
:1012d0000100fc000108a900ff3ffc003200f900fa
:1012e000ae0120000d0009004f1778004f0778006d
:1012f0004400f9003600f9004200f9000100fc004a
:1013000000400600ff3ffc004200f8003600f800f5
:101310004400f8008e1f78000e0020000d00090028
:10132000be1f78003200f8000100fc000368a9002d
:101330001421ef00ff3ffc003200f900ae01200055
:101340000d0009004f1778004f0778004400f9009e
:101350003600f9004200f9000100fc0000400600e0
:10136000ff3ffc004200f8003600f8004400f8009f
:101370008e1f78000e0020000d000900be1f7800af
:101380003200f8000100fc000388a9001821ef00da
:101390002023a800ff3ffc003200f900ae0120002e
:1013a0000d0009004f1778004f0778004400f9003e
:1013b0003600f9004200f9000100fc000040060080
:1013c000ff3ffc004200f8003600f8004400f8003f
:1013d0008e1f78000e0020000d000900be1f78004f
:1013e0003200f8000100fc000168a9004a72ec001c
:1013f0004ad2bf008080fb0030118000c2762100fd
:1014000080707900ff3ffc003200f900ae0120003f
:101410000d0009004f1778004f0778004400f900cd
:101420003600f9004200f9000100fc00004006000f
:10143000ff3ffc004200f8003600f8004400f800ce
:101440008e1f78000e0020000d000900be1f7800de
:101450003200f8000100fc000828a9002242ae007a
:10146000000037002222af002222a900ff3ffc002b
:101470003200f900ae0120000d0009004f1778007e
:101480004f0778004400f9003600f9004200f900e7
:101490000100fc0000400600ff3ffc004200f80095
:1014a0003600f8004400f8008e1f78000e0020007f
:1014b0000d000900be1f78003200f8000100fc009a
:1014c0000188a900ff3ffc003200f900ae012000b6
:1014d0000d0009004f1778004f0778004400f9000d
:1014e0003600f9004200f9000100fc00004006004f
:1014f000ff3ffc004200f8003600f8004400f8000e
:101500008e1f78000e0020000d000900be1f78001d
:101510003200f8000100fc0000188000a091880053
:1015200001a8a9002003a900ff3ffc003200f90038
:10153000ae0120000d0009004f1778004f0778001a
:101540004400f9003600f9004200f9000100fc00f7
:1015500000400600ff3ffc004200f8003600f800a3
:101560004400f8008e1f78000e0020000d000900d6
:10157000be1f78003200f8000100fc000bc8a90073
:10158000ff3ffc003200f900ae0120000d00090011
:101590004f1778004f0778004400f9003600f90033
:1015a0004200f9000100fc0000400600ff3ffc0083
:1015b0004200f8003600f8004400f8008e1f780062
:1015c0000e0020000d000900be1f78003200f80058
:1015d0000100fc000be8a900ff3ffc003200f9000d
:1015e000ae0120000d0009004f1778004f0778006a
:1015f0004400f9003600f9004200f9000100fc0047
:1016000000400600ff3ffc004200f8003600f800f2
:101610004400f8008e1f78000e0020000d00090025
:10162000be1f78003200f8000100fc000c08a90081
:10163000ff3ffc003200f900ae0120000d00090060
:101640004f1778004f0778004400f9003600f90082
:101650004200f9000100fc00004006004bd2bf0030
:101660004a52e300070032004b72ec004bd2bf003d
:101670000080fb00c176210060c078004cf2b7000a
:10168000010037004cf2ef00000006005008800017
:10169000c091880030088000b0918800efff0700fb
:1016a000e0ceb3004c52b50006003900e0cfb300e5
:1016b0004c52b50001003900010037004d72ef00b7
:1016c0000f0137004cf2ae00370037004d72ef00cb
:1016d000d0c8b3004c52e30005003a004cd2bf0022
:1016e0004df2b7004ef2ef004ff2ef002d00370041
:1016f000d0c9b3004c52e30005003a004cd2bf0001
:101700004df2b70050f2ef0051f2ef002500370024
:10171000d0cab3004c52e30005003a004cd2bf00df
:101720004df2b70052f2ef0053f2ef001d00370008
:10173000d0cbb3004c52e30005003a004cd2bf00be
:101740004df2b70054f2ef0055f2ef0015003700ec
:10175000d0ccb3004c52e30004003a004cd2bf009e
:101760004df2b70056f2ef000e003700d0cdb300b7
:101770004c52e30004003a004cd2bf004df2b700d7
:1017800057f2ef0007003700d0ceb3004c52e30011
:1017900004003a004cd2bf004df2b70058f2ef00ff
:1017a00059f2ef00d60037004d52e20002003a0035
:1017b000d3003700d2003700d0c8b3004d52e30049
:1017c00038003a0000e0ef004e52e30003003a0018
:1017d0004cd2bf004ef2b700310037004cd2bf00f0
:1017e0004ff2b70080c1b3004e52e3002b003a0025
:1017f0004f52e20012003a0014cea90005e1a90000
:101800000008200030618800000820003062880055
:1018100000082000306388006472ef003212a900d3
:101820002812ae000400370068b7ef006ab7ef0077
:101830005c12a8002812a900140ea9001700370096
:10184000022eae00150037003212a80005e1a800f4
:10185000028020004fd2bf000080fb000200b800d1
:101860000001be0042bb880053bb880042bb800021
:1018700053bb8000b0918000c19180000200400005
:10188000838048000001be0042bb880053bb880033
:101890002812a8005c12a800140ea9004ef2ef0056
:1018a00097003700d0c9b3004d52e30044003a001e
:1018b00000e0ef005052e30003003a004cd2bf00ba
:1018c00050f2b7003d0037004cd2bf0051f2b700d4
:1018d0005152e20014003a0080c1b3005052e300bc
:1018e00010003a0014cea90005e1a900000820006c
:1018f0003061880000082000306288000008200065
:10190000306388003212a9002812ae0004003700ac
:1019100068b7ef006ab7ef005c12a8002812a900b0
:10192000140ea9002400370080c1b3005052e30018
:1019300021003a0051d2bf0065f2b700022eae007e
:101940001900370065d2bf000080fb000000400096
:1019500081262100608078001008880005e1a80039
:101960000068a9002068a80065d2bf000080fb00c5
:101970004200de00010220000080500064f2b70047
:101980003212a9002812ae000400370068b7ef0039
:101990006ab7ef005c12a8002812a90014cea800b4
:1019a000140ea8000400370014cea900140ea900dc
:1019b00000c2b30064f2b70050f2ef0050003700ed
:1019c000d0cab3004d52e3001f003a0000e0ef0020
:1019d0005252e30003003a004cd2bf0052f2b7006b
:1019e000180037004cd2bf0053f2b70080c1b300db
:1019f0005252e30012003a0012ceae00100037003f
:101a000010cea90014cea8003212af000c0037008f
:101a100053d2bf000080fb004200de000102200024
:101a20000080500064f2b70053d2bf000080fb007a
:101a300000004000812621006080780010088800a6
:101a400052f2ef002e003700d0cbb3004d52e3002e
:101a50000b003a0000e0ef005452e30003003a00ac
:101a60004cd2bf0054f2b700040037004cd2bf0084
:101a700055f2b7003601070054f2ef00200037009e
:101a8000d0ccb3004d52e30007003a0000e0ef0075
:101a90005652e30003003a004cd2bf0056f2b700a2
:101aa00056f2ef0016003700d0cdb3004d52e300e0
:101ab00007003a0000e0ef005752e30003003a004d
:101ac0004cd2bf0057f2b70057f2ef000c003700be
:101ad000d0ceb3004d52e30009003a0000e0ef0021
:101ae0005852e30003003a004cd2bf0058f2b7004e
:101af000030037004cd2bf0059f2b70058f2ef0094
:101b0000022eaf00490037000100200037f2af007d
:101b10001140b0006612af001140b1004300320026
:101b20006612a80037f2ae006612a900a0918000ec
:101b30004500de0067f2b7006752e2002900360078
:101b40006632af001800370067d2bf000080fb008c
:101b50000000400081262100608078001008880085
:101b600005e1a8000068a9002068a80067d2bf00ae
:101b70000080fb004200de000102200000805000d7
:101b800064f2b7003212a9002812ae000400370038
:101b900068b7ef006ab7ef005c12a8002812a9002e
:101ba0006632a8000c00370067d2bf000080fb003f
:101bb0000000400081262100608078001008880025
:101bc00067d2bf000080fb004200de00010220005f
:101bd0000080500064f2b70014cea800140ea800d4
:101be0001200370014cea90005e1a900000820006a
:101bf0003061880000082000306288000008200062
:101c0000306388006472ef003212a9002812ae001f
:101c10000400370068b7ef006ab7ef005c12a80055
:101c20002812a900140ea9006632a9005c12af00a8
:101c3000aa00070010c0b3005b52b50026003100b7
:101c4000b2918000c3918000f091800001928000e9
:101c5000800f5100818f59001300390041f2a80014
:101c60005b52e2000f003a0014cea90005e1a90082
:101c700000082000306188000008200030628800e1
:101c8000000820003063880000c2b30064f2b7008f
:101c900068b7ef006ab7ef003212a9002812a90056
:101ca0006632a9008d00070039f2ae000900370046
:101cb0000621ef000a21ef003632ef003832ef0044
:101cc0000080eb0081762100010009008018780077
:101cd0006efe37000400370039f2ae000200370014
:101ce0000621ef000a21ef005dd2bf005e52e30043
:101cf000750032002068a9003212af0037003700ab
:101d000064d2bf005e52b40061f2b7005ed2bf0081
:101d10000080fb00000040008136210060807800d8
:101d2000d090880061d2bf000080fb00000040001e
:101d300081362100608078001a12b400509188002a
:101d40005ed2bf005041b0005ff2b70064d2bf0066
:101d50005f52b40062f2b7005fd2bf000080fb00a8
:101d6000000040008136210060807800d09088001b
:101d700062d2bf000080fb000000400081362100dd
:101d8000608078001a12b400609188005ed2bf00b3
:101d9000b042b00060f2b70064d2bf006052b4003d
:101da00063f2b70060d2bf000080fb00000040007b
:101db0008136210060807800d090880063d2bf0017
:101dc0000080fb0000004000813621006080780028
:101dd0001a12b40070918800380037002812ae0043
:101de000300037005ed2bf000080fb0000004000e2
:101df0008136210060807800d09088005ed2bf00dc
:101e00000080fb00000040008136210060807800e7
:101e10001a12b4005091880050c1b3005e52b50050
:101e20005ff2b7005fd2bf000080fb0000004000ff
:101e30008136210060807800d09088005fd2bf009a
:101e40000080fb00000040008136210060807800a7
:101e50001a12b40060918800b0c2b3005e52b5009f
:101e600060f2b70060d2bf000080fb0000004000bd
:101e70008136210060807800d090880060d2bf0059
:101e80000080fb0000004000813621006080780067
:101e900000918800d09080002012bc0072918800d0
:101ea000060037000000280050918800000028003c
:101eb0006091880000002800709188005ed2bf0009
:101ec0005df2b7002068a8003832af0014aea80059
:101ed0003832ae0014aea900ecfd37005bf2ef0023
:101ee00041f2a8002632ef0030918000c200dd00f0
:101ef00080762100008040001000be000001be007e
:101f0000f091800001928000800f5100818f590074
:101f10000900310030918000c200dd008076210090
:101f2000008040001000be00f091880001928800ff
:101f300026d2bf005bf2b7002632ec003191800060
:101f4000e18f5000e8ff3a005c12a9000000060093
:101f500020c4b3005452e3001c003a005552e20082
:101f600018003a002632ef002612e20009003e0077
:101f700030918000c200dd008076210000814000a9
:101f8000f0ff2f00f1ff2f000089be002632ec0089
:101f9000f5ff390005e1a9002832ef005c12a80026
:101fa00014cea900042ea90000082000306188008a
:101fb000000820003062880000082000306388009c
:101fc00001003700042ea8000d003700b0c7b30091
:101fd0005452e3000a003a0014cea9000008200081
:101fe000306188000008200030628800000820006e
:101ff0003063880068b7ef006ab7ef002832ef005f
:1020000054f2ef000000060068b6ef00101a2f002f
:1020100050b3880010412e0060b3880040742d003a
:1020200070b38800f0b22c0080b3880070fc2b00e5
:1020300090b3880030502b00a0b38800a0ad2a00d8
:10204000b0b3880030142a00c0b388006083290030
:10205000d0b38800b0fa2800e0b38800a079280047
:10206000f0b38800c00020003091880031918000da
:10207000f78f50000e003e00c00020002612b50071
:10208000000678000c0646008066210060007e0095
:102090004100de00329180004111dd0081662100a7
:1020a00001014100000978002632ec00efff390001
:1020b00080012000309188003191800030022000a2
:1020c000808f50000e003e00800120002612b500d7
:1020d000000678000c0646008066210060007e0045
:1020e0004200de00329180004111dd008166210056
:1020f00001014100000978002632ec00eeff3900b2
:10210000400220003091880031918000f0022000d0
:10211000808f50000e003e00400220002612b500c5
:10212000000678000c0646008066210060007e00f4
:102130004300de00329180004111dd008166210004
:1021400001014100000978002632ec00eeff390061
:10215000000320003091880031918000b0032000fe
:10216000808f50000e003e00000320002612b500b4
:10217000000678000c0646008066210060007e00a4
:102180004400de00329180004111dd0081662100b3
:1021900001014100000978002632ec00eeff390011
:1021a000c00320003091880031918000700420002d
:1021b000808f50000e003e00c00320002612b500a4
:1021c000000678000c0646008066210060007e0054
:1021d0004500de00329180004111dd008166210062
:1021e00001014100000978002632ec00eeff3900c1
:1021f000800420003091880031918000300520005b
:10220000808f50000e003e00800420002612b50092
:10221000000678000c0646008066210060007e0003
:102220004600de00329180004111dd008166210010
:1022300001014100000978002632ec00eeff390070
:10224000007a210080b88800f073210090b88800df
:10225000f06d2100a0b8880000682100b0b88800a7
:1022600040622100c0b88800805c2100d0b888009e
:10227000e0562100e0b8880060512100f0b88800e5
:10228000f04b210000b988009046210010b9880069
:102290005041210020b98800203c210030b988003d
:1022a0001037210040b988001032210050b9880051
:1022b000202d210060b988004028210070b98800d5
:1022c0008023210080b98800d01e210090b98800a9
:1022d000301a2100a0b98800a0152100b0b98800eb
:1022e00020112100c0b98800c00c2100d0b988009d
:1022f00070082100e0b9880020042100f0b98800ae
:10230000f0ff200000ba8800d0fb200010ba88003f
:10231000c0f7200020ba8800d0f3200030ba88002f
:10232000e0ef200040ba880000ec200050ba88009e
:1023300030e8200060ba880070e4200070ba88009d
:10234000c0e0200080ba880020dd200090ba88001c
:1023500090d92000a0ba880010d62000b0ba88001a
:10236000a0d22000c0ba880040cf2000d0ba880098
:10237000e0cb2000e0ba8800a0c82000f0ba8800b6
:1023800060c5200000bb880030c2200010bb880060
:1023900010bf200020bb880000bc200030bb88009c
:1023a0000000060068b5ef00a0c7250050ab88000c
:1023b0005098250060ab88004081250070ab8800f4
:1023c000906a250080ab88003054250090ab8800cf
:1023d000303e2500a0ab880090282500b0ab8800d7
:1023e00050132500c0ab880060fe2400d0ab8800ed
:1023f000c0e92400e0ab880080d52400f0ab880061
:1024000090c1240000ac8800f0ad240010ac88001e
:10241000a09a240020ac8800a087240030ac88005b
:10242000f074240040ac88009062240050ac880016
:102430008050240060ac8800b03e240070ac88005e
:10244000302d240080ac8800f01b240090ac880064
:10245000000b2400a0ac880050fa2300b0ac880028
:10246000e0e92300c0ac8800c0d92300d0ac8800cc
:10247000e0c92300e0ac880040ba2300f0ac88003b
:10248000e0aa230000ad8800c09b230010ad8800a7
:10249000e08c230020ad8800307e230030ad880022
:1024a000d06f230040ad8800a061230050ad8800ac
:1024b000b053230060ad8800f045230070ad880064
:1024c0007038230080ad8800202b230090ad880059
:1024d000101e2300a0ad880040112300b0ad88007d
:1024e00090042300c0ad880020f82200d0ad880001
:1024f000e0eb2200e0ad8800d0df2200f0ad8800e4
:10250000f0d3220000ae880050c8220010ae880030
:10251000d0bc220020ae880080b1220030ae8800fe
:1025200070a6220040ae8800809b220050ae88003a
:10253000c090220060ae88002086220070ae880025
:10254000c07b220080ae88008071220090ae88009f
:1025500060672200a0ae8800805d2200b0ae8800d7
:10256000c0532200c0ae8800204a2200d0ae8800ae
:10257000b0402200e0ae880060372200f0ae880054
:10258000402e220000af88004025220010af8800b6
:10259000601c220020af8800b013220030af8800fa
:1025a000200b220040af8800b002220050af88000c
:1025b00060fa210060af880040f2210070af88000f
:1025c00030ea210080af880050e2210090af8800ff
:1025d00090da2100a0af8800e0d22100b0af8800df
:1025e00060cb2100c0af8800f0c32100d0af8800cd
:1025f000b0bc2100e0af880080b52100f0af8800ba
:1026000080ae210000b0880090a7210010b08800a3
:10261000b0a0210020b08800009a210030b08800ce
:102620006093210040b08800e08c210050b0880009
:102630008086210060b088003080210070b0880062
:10264000007a210080b08800f073210090b08800eb
:10265000f06d2100a0b0880000682100b0b08800b3
:1026600040622100c0b08800805c2100d0b08800aa
:10267000e0562100e0b0880060512100f0b08800f1
:10268000f04b210000b188009046210010b1880075
:102690005041210020b18800203c210030b1880049
:1026a0001037210040b188001032210050b188005d
:1026b000202d210060b188004028210070b18800e1
:1026c0008023210080b18800d01e210090b18800b5
:1026d000301a2100a0b18800a0152100b0b18800f7
:1026e00020112100c0b18800c00c2100d0b18800a9
:1026f00070082100e0b1880020042100f0b18800ba
:10270000f0ff200000b28800d0fb200010b288004b
:10271000c0f7200020b28800d0f3200030b288003b
:10272000e0ef200040b2880000ec200050b28800aa
:1027300030e8200060b2880070e4200070b28800a9
:10274000c0e0200080b2880020dd200090b2880028
:1027500090d92000a0b2880010d62000b0b2880026
:10276000a0d22000c0b2880040cf2000d0b28800a4
:10277000e0cb2000e0b28800a0c82000f0b28800c2
:1027800060c5200000b3880030c2200010b388006c
:1027900010bf200020b3880000bc200030b38800a8
:1027a0000000060090dc230020928800b0fd20008d
:1027b000109288002632ef0027f2bf0019003a007d
:1027c000129280002392800030918000d7f8070099
:1027d0005df8070023f707003092880041928800d7
:1027e00032928000439280000000200001f8230014
:1027f000f7f707000001be0000c02f00f1672400ba
:1028000051f80700aaf80700329180004111dd005d
:102810008136210001014100000978002632ec00d8
:10282000e5ff39000000060040122000309b8800c0
:10283000c0122000209b880060132000109b88009d
:10284000b0132000009b880000142000f09a88003c
:1028500050142000e09a8800b0142000d09a88001c
:1028600000152000c09a880060152000b09a8800ea
:10287000b0152000a09a880010162000909a8800b9
:1028800070162000809a8800d0162000709a880068
:1028900030172000609a880090172000509a880016
:1028a000f0172000409a880050182000309a8800c5
:1028b000b0182000209a880020192000109a880063
:1028c00080192000009a8800f0192000f0998800f3
:1028d000601a2000e0998800d01a2000d099880062
:1028e000401b2000c0998800b01b2000b0998800d0
:1028f000201c2000a0998800a01c2000909988002e
:10290000101d200080998800901d2000709988007b
:10291000101e200060998800801e200050998800b9
:10292000001f200040998800901f200030998800e7
:102930001020200020998800902020001099880005
:102940002021200000998800a0212000f098880014
:1029500030222000e0988800c0222000d098880013
:1029600050232000c0988800f0232000b0988800f1
:1029700080242000a09888002025200090988800be
:10298000b02520008098880050262000709888008c
:10299000f02620006098880090272000509888003a
:1029a0004028200040988800e028200030988800c7
:1029b0009029200020988800402a20001098880044
:1029c000f02a200000988800a02b2000f0978800b3
:1029d000602c2000e0978800102d2000d097880000
:1029e000d02d2000c0978800902e2000b09788003e
:1029f000502f2000a097880020302000909788005a
:102a0000e030200080978800b03120007097880067
:102a10008032200060978800503320005097880053
:102a2000303420004097880010352000309788000f
:102a3000e035200020978800d036200010978800cd
:102a4000b03720000097880090382000f09688006a
:102a500080392000e0968800703a2000d0968800e7
:102a6000703b2000c0968800603c2000b096880033
:102a7000603d2000a0968800603e2000909688006f
:102a8000703f20008096880070402000709688007b
:102a90008041200060968800904220005096880077
:102aa000b043200040968800c04420003096880043
:102ab000e0452000209688001047200010968800ee
:102ac000304820000096880060492000f09588007a
:102ad000a04a2000e0958800d04b2000d0958800c7
:102ae000104d2000c0958800504e2000b095880001
:102af000a04f2000a0958800f050200090958800fd
:102b000040522000809588009053200070958800e6
:102b1000f0542000609588005056200050958800a1
:102b2000c05720004095880030592000309588001b
:102b3000a05a200020958800205c20001095880075
:102b4000a05d200000958800305f2000f094880090
:102b5000c0602000e094880050622000d09488007b
:102b6000f0632000c094880090652000b094880035
:102b700040672000a0948800f068200090948800ae
:102b8000a06a200080948800606c20007094880007
:102b9000306e200060948800f06f20005094880010
:102ba000d071200040948800b073200030948800d9
:102bb0009075200020948800807720001094880071
:102bc0007079200000948800707b2000f0938800ca
:102bd000707d2000e0938800807f2000d0938800e3
:102be000a0812000c0938800c0832000b09388009b
:102bf000e0852000a0938800108820009093880032
:102c0000508a200080938800908c20007093880068
:102c1000e08e20006093880030912000509388005f
:102c2000909320004093880000000600ffff3700cb
:020000040000fa
:102c30001a1200000c0000008000000026120000a4
:102c40001000000080000000361200001400000098
:102c5000800000004a1200001e00000080000000fa
:102c600068120000000500008000000068170000e6
:102c700004000000800000006c170000000100004c
:082c80008000000000000000cc
:00000001FF
